:05000000020033E1895C
:02000B00E18A88
:02001300E18B7F
:02001B00E18C76
:02002300E18D6D
:02002B00E18E64
:10003300759840758780758921758DFF758BFF7560
:100043008840D2997581077530007531007535FF89
:10005300D210D211D212D213D214D215D216D21771
:10006300D218D219D21AD21BD21CD21DD21ED21F21
:10007300D234D235D236D237C2B0741FB5350375F8
:1000830035FF0535E535A2E092A4A2E192A5A2E2EF
:1000930092A6A2E392A7A2E492A1B392A2D2A3D280
:1000A30090209014301021C210B2112011051207B4
:1000B300A980151207C9801020100DD21020110538
:1000C3001207C580031207E5C2A3D2912091143011
:1000D3001221C212B2132013051207E98015120868
:1000E30009801020120DD212201305120805800377
:1000F300120825D292209214301421C214B2152072
:1001030015051208298015120849801020140DD2F4
:10011300142015051208458003120865D293209315
:1001230014301621C216B21720170512086980155C
:10013300120889801020160DD21620170512088583
:1001430080031208A5D294209414301821C218B247
:10015300192019051208A980151208C98010201842
:100163000DD2182019051208C580031208E5D2958F
:10017300209514301A21C21AB21B201B051208E95C
:1001830080151209098010201A0DD21A201B05129E
:1001930009058003120925D296209614301C21C22A
:1001A3001CB21D201D051209298015120949801052
:1001B300201C0DD21C201D05120945800312096560
:1001C300D297209714301E21C21EB21F201F051282
:1001D300096980151209898010201E0DD21E201F67
:1001E3000512098580031209A5D2B220B214303456
:1001F30021C234B2352035051209A980151209D15F
:10020300801020340DD2342035051209CD8003121D
:1002130009F5D2B320B314303621C236B2372037B2
:10022300051209F98015120A19801020360DD236ED
:10023300203705120A158003120A35D2B420B41CE4
:10024300753207120A3912078FD532067532011239
:100253000A39120796D2B420B40280EDD2B520B584
:100263001C753207120A5712078FD53206753201F1
:10027300120A57120796D2B520B50280EDD2B620E6
:10028300B61C753207120A7512078FD532067532FE
:1002930001120A75120796D2B620B60280EDD2B7C4
:1002A30020B71C753207120A8E12078FD5320675D6
:1002B3003201120A8E120796D2B720B70280EDE4FC
:1002C300B53502618404B5350261A404B535026114
:1002D300C404B5350261E404B53502810404B535BF
:1002E30002812404B53502814404B53502816404D6
:1002F300B53502818404B5350281A404B535028184
:10030300C404B5350281E404B53502A10404B5354E
:1003130002A12404B53502A14404B53502A1640445
:10032300B53502A18404B53502A1A404B53502A1F3
:10033300C404B53502A1E404B53502C10404B535DE
:1003430002C12404B53502C14404B53502C16404B5
:10035300B53502C18404B53502C1A404B53502C163
:10036300C404B53502C1E404B53502E10404B5356E
:1003730002E12404B53502E14404B53502E164E148
:1003830084E580F536A837A93612079D400624FE7A
:10039300500D80051207A25006853637120AA7E1D1
:1003A30084E580F538A839A93812079D400624FE54
:1003B300500D80051207A25006853839120AC3E191
:1003C30084E580F53AA83BA93A12079D400624FE2E
:1003D300500D80051207A25006853A3B120ADFE151
:1003E30084E580F53CA83DA93C12079D400624FE08
:1003F300500D80051207A25006853C3D120AFBE111
:1004030084E580F53EA83FA93E12079D400624FEE1
:10041300500D80051207A25006853E3F120B17E1CF
:1004230084E580F540A841A94012079D400624FEBB
:10043300500D80051207A25006854041120B33E18F
:1004430084E580F542A843A94212079D400624FE95
:10045300500D80051207A25006854243120B4FE14F
:1004630084E580F544A845A94412079D400624FE6F
:10047300500D80051207A25006854445120B6BE10F
:1004830084E580F546A847A94612079D400624FE49
:10049300500D80051207A25006854647120B87E1CF
:1004A30084E580F548A849A94812079D400624FE23
:1004B300500D80051207A25006854849120BA3E18F
:1004C30084E580F54AA84BA94A12079D400624FEFD
:1004D300500D80051207A25006854A4B120BBFE14F
:1004E30084E580F54CA84DA94C12079D400624FED7
:1004F300500D80051207A25006854C4D120BDBE10F
:1005030084E580F54EA84FA94E12079D400624FEB0
:10051300500D80051207A25006854E4F120BF7E1CE
:1005230084E580F550A851A95012079D400624FE8A
:10053300500D80051207A25006855051120C13E18D
:1005430084E580F552A853A95212079D400624FE64
:10055300500D80051207A25006855253120C2FE14D
:1005630084E580F554A855A95412079D400624FE3E
:10057300500D80051207A25006855455120C4BE10D
:1005830084E580F556A857A95612079D400624FE18
:10059300500D80051207A25006855657120C67E1CD
:1005A30084E580F558A859A95812079D400624FEF2
:1005B300500D80051207A25006855859120C83E18D
:1005C30084E580F55AA85BA95A12079D400624FECC
:1005D300500D80051207A25006855A5B120C9FE14D
:1005E30084E580F55CA85DA95C12079D400624FEA6
:1005F300500D80051207A25006855C5D120CBBE10D
:1006030084E580F55EA85FA95E12079D400624FE7F
:10061300500D80051207A25006855E5F120CD7E1CC
:1006230084E580F560A861A96012079D400624FE59
:10063300500D80051207A25006856061120CF3E18C
:1006430084E580F562A863A96212079D400624FE33
:10065300500D80051207A25006856263120D0FE14B
:1006630084E580F564A865A96412079D400624FE0D
:10067300500D80051207A25006856465120D2BE10B
:1006830084E580F566A867A96612079D400624FEE7
:10069300500D80051207A25006856667120D47E1CB
:1006A30084E580F568A869A96812079D400624FEC1
:1006B300500D80051207A25006856869120D63E18B
:1006C30084E580F56AA86BA96A12079D400624FE9B
:1006D300500D80051207A25006856A6B120D7FE14B
:1006E30084E580F56CA86DA96C12079D400624FE75
:1006F300500D80051207A25006856C6D120D9BE10B
:1007030084E580F56EA86FA96E12079D400624FE4E
:10071300500D80051207A25006856E6F120DB7E1CA
:1007230084E580F570A871A97012079D400624FE28
:10073300500D80051207A25006857071120DD3E18A
:1007430084E580F572A873A97212079D400624FE02
:10075300500D80051207A25006857273120DEFE14A
:1007630084E580F574A875A97412079D400624FEDC
:10077300500D80051207A25006857475120E0BE109
:1007830084017B0200333232323232327E20DFFE8A
:10079300DEFC227E60DFFEDEFC22C2D7E89922C2A5
:1007A300D7E99824FE223099FDC2997599B0309902
:1007B300FDC2997599663099FDC29975997F1207A3
:1007C3008F2212078F223099FDC2997599B0309903
:1007D300FDC2997599663099FDC29975997F120783
:1007E3008F2212078F223099FDC2997599B03099E3
:1007F300FDC2997599673099FDC29975997F120762
:100803008F2212078F223099FDC2997599B03099C2
:10081300FDC2997599673099FDC29975997F120741
:100823008F2212078F223099FDC2997599B03099A2
:10083300FDC2997599683099FDC29975997F120720
:100843008F2212078F223099FDC2997599B0309982
:10085300FDC2997599683099FDC29975997F120700
:100863008F2212078F223099FDC2997599B0309962
:10087300FDC2997599693099FDC29975997F1207DF
:100883008F2212078F223099FDC2997599B0309942
:10089300FDC2997599693099FDC29975997F1207BF
:1008A3008F2212078F223099FDC2997599B0309922
:1008B300FDC29975996A3099FDC29975997F12079E
:1008C3008F2212078F223099FDC2997599B0309902
:1008D300FDC29975996A3099FDC29975997F12077E
:1008E3008F2212078F223099FDC2997599B03099E2
:1008F300FDC29975996B3099FDC29975997F12075D
:100903008F2212078F223099FDC2997599B03099C1
:10091300FDC29975996B3099FDC29975997F12073C
:100923008F2212078F223099FDC2997599B03099A1
:10093300FDC29975996C3099FDC29975997F12071B
:100943008F2212078F223099FDC2997599B0309981
:10095300FDC29975996C3099FDC29975997F1207FB
:100963008F2212078F223099FDC2997599B0309961
:10097300FDC29975996D3099FDC29975997F1207DA
:100983008F2212078F223099FDC2997599B0309941
:10099300FDC29975996D3099FDC29975997F1207BA
:1009A3008F2212078F22E53004B40801E4F53030BA
:1009B30099FDC2997599B03099FDC29975997030B6
:1009C30099FDC299F59912078F2212078F22E530FC
:1009D30004B40801E4F5303099FDC2997599B0303B
:1009E30099FDC2997599703099FDC299F5991207CD
:1009F3008F2212078F223099FDC2997599B03099D1
:100A0300FDC2997599713099FDC29975997F120745
:100A13008F2212078F223099FDC2997599B03099B0
:100A2300FDC2997599713099FDC2997599001207A4
:100A33008F2212078F223099FDC2997599B0309990
:100A4300FDC2997599723099FDC2990531E531540A
:100A53007FF599223099FDC2997599B03099FDC2FD
:100A6300997599723099FDC2991531E531547FF525
:100A730099223099FDC2997599B03099FDC2997543
:100A830099733099FDC29975997F223099FDC29966
:100A93007599B03099FDC2997599743099FDC299D1
:100AA30075997F223099FDC2997599B03099FDC22D
:100AB300997599003099FDC299E536C313F59922CA
:100AC3003099FDC2997599B03099FDC29975990114
:100AD3003099FDC299E538C313F599223099FDC2C7
:100AE300997599B03099FDC2997599023099FDC2F3
:100AF30099E53AC313F599223099FDC2997599B0D6
:100B03003099FDC2997599033099FDC299E53CC3AB
:100B130013F599223099FDC2997599B03099FDC2A8
:100B2300997599043099FDC299E53EC313F599224D
:100B33003099FDC2997599B03099FDC2997599059F
:100B43003099FDC299E540C313F599223099FDC24E
:100B5300997599B03099FDC2997599063099FDC27E
:100B630099E542C313F599223099FDC2997599B05D
:100B73003099FDC2997599073099FDC299E544C32F
:100B830013F599223099FDC2997599B03099FDC238
:100B9300997599083099FDC299E546C313F59922D1
:100BA3003099FDC2997599B03099FDC2997599092B
:100BB3003099FDC299E548C313F599223099FDC2D6
:100BC300997599B03099FDC29975990A3099FDC20A
:100BD30099E54AC313F599223099FDC2997599B0E5
:100BE3003099FDC29975990B3099FDC299E54CC3B3
:100BF30013F599223099FDC2997599B03099FDC2C8
:100C03009975990C3099FDC299E54EC313F5992254
:100C13003099FDC2997599B03099FDC29975990DB6
:100C23003099FDC299E550C313F599223099FDC25D
:100C3300997599B03099FDC29975990E3099FDC295
:100C430099E552C313F599223099FDC2997599B06C
:100C53003099FDC29975990F3099FDC299E554C336
:100C630013F599223099FDC2997599B03099FDC257
:100C7300997599103099FDC299E556C313F59922D8
:100C83003099FDC2997599B03099FDC29975991142
:100C93003099FDC299E558C313F599223099FDC2E5
:100CA300997599B03099FDC2997599123099FDC221
:100CB30099E55AC313F599223099FDC2997599B0F4
:100CC3003099FDC2997599133099FDC299E55CC3BA
:100CD30013F599223099FDC2997599B03099FDC2E7
:100CE300997599143099FDC299E55EC313F599225C
:100CF3003099FDC2997599B03099FDC299759915CE
:100D03003099FDC299E560C313F599223099FDC26C
:100D1300997599B03099FDC2997599163099FDC2AC
:100D230099E562C313F599223099FDC2997599B07B
:100D33003099FDC2997599173099FDC299E564C33D
:100D430013F599223099FDC2997599B03099FDC276
:100D5300997599183099FDC299E566C313F59922DF
:100D63003099FDC2997599B03099FDC29975991959
:100D73003099FDC299E568C313F599223099FDC2F4
:100D8300997599B03099FDC29975991A3099FDC238
:100D930099E56AC313F599223099FDC2997599B003
:100DA3003099FDC29975991B3099FDC299E56CC3C1
:100DB30013F599223099FDC2997599B03099FDC206
:100DC3009975991C3099FDC299E56EC313F5992263
:100DD3003099FDC2997599B03099FDC29975991DE5
:100DE3003099FDC299E570C313F599223099FDC27C
:100DF300997599B03099FDC29975991E3099FDC2C4
:100E030099E572C313F599223099FDC2997599B08A
:100E13003099FDC29975991F3099FDC299E574C344
:100E230013F59922204D757A796B616E7420382001
:100E330076312E306220323030372D31322D31353C
:100E4300202863294164616D20536D69616C656B72
:100E5300206A616E6B6F6D757A796B616E74407722
:100E6300702E706C207777772E736D69616C656B6C
:100E73002E7072762E706C2057737A656C6B696571
:100E8300207072617761207A617374727A657A6F08
:100E93006E652E204A616B69656B6F6C7769656B54
:100EA300207A6173746F736F77616E6961206B6F02
:100EB3006D657263796A6E65206B6F6475206E6908
:100EC30065646F7A776F6C6F6E652E20416C6C2052
:100ED3005269676874732052657365727665642E10
:100EE300204672656520666F72206E6F6E20636F99
:0F0EF3006D6D65726369616C206F6E6C792E2076
:00000001FF
